:0200000080245A
:080003000210030000000000E0
:08000B0002100B0000000000D0
:080013000210130000000000C0
:08001B0002101B0000000000B0
:10002300021023E4F5D0F50EF50D758130538EFEE5
:1000330053A23FF13930B050C28E75985A75892159
:10004300758D00789020B0FDD8FE158D785E30B0A8
:10005300F720B0FD30B0FDD28E758DFD758BFD316F
:10006300000D4D43532D35312054494E5920424103
:100073005349432F415320544235314D4C323420A0
:1000830056322E348D02088BD242D2410208AC3054
:1000930098FDE599C298547FB403022129B4610005
:1000A3004007B47B00500254DF22740D3099FDC227
:1000B30099F599B40D0A3099FDC29975990A80048E
:1000C300C3D52B04752B08D32230980A1192B4138D
:1000D300051192B411FB22742011AF50FA22540F70
:1000E3007003204807C24824038311AF2230313202
:1000F30033343536373839414243444546D083D0CB
:1001030082E493A310E70411AF80F611AFE4730206
:10011300088E3100484F573F8D80F43100534F52C2
:100123005259218D80E931000D574841543F8D804C
:10013300DEA980B982004021FEE7FF19E7CE1989C5
:10014300801922A980E7158022A980B9D900500916
:1001530009EEF709EFF7898022311E0FA980B9D97B
:100163000050F619E70987F009F709A7F0898022FB
:10017300D083D082E4930580A980B9DB02809CF709
:100183007401D3738090A0B08898A8B8898A8B8CA7
:100193008D998E80228E90228EA0228EB0228E8800
:1001A300228E98228EA8228EB8228E89228E8A22AF
:1001B3008E8B228E8C228E8D228E9922E58022E5D3
:1001C3009022E5A022E5B022E58822E59822E5A861
:1001D30022E5B822E58922E58A22E58B22E58C22F5
:1001E300E58D22E59922900187E4FDED9369700482
:1001F300ED232D220DEDB40EF22115FEE920E703C8
:10020300EEF72231E990019573E920E702E7223105
:10021300E99001BF73EE54F820E70423C42420F9C6
:10022300EE5407240383F5F0220102040810204052
:1002330080D24B8002C24B31348E088F0931343166
:1002430046304B0605800580058090025293730566
:10025300252B4040EE2320400D2410F924D940994A
:10026300A70809A70922F582758300E508F005822E
:10027300E509F022EEF9E50880815118510CFEE5FD
:100283000820E006E5F0F45E21FEE5F04E21FE8F46
:10029300838E82E508F022D24B8002C24B31343187
:1002A30046304B060580058005809002B2937305A6
:1002B300272D3940EE2320400E2410F924D9401471
:1002C300E7FE09E7FF214CF582758300E0FE058216
:1002D300E0FF214C21FCEEF9510C80195118510C0F
:1002E30055F024FFE433800D8F838E82E080068FE8
:1002F300838E82E4937F00FE214C24D0B40A005005
:1003030005FE7F00C24D22204D3E24D0B40A00409A
:100313001330443424EFB406004007B4072AD24D07
:10032300D322240ACE75F00A30440375F010C0F0CE
:10033300A42EFEE435F0CFD0F0A42FFF72E7E5F052
:1003430034FFB0444004D322C322311502A2D2B0F9
:1003530044400122311506E72EF709E73FF7223122
:1003630034715A80E83134C3E79EF709E79FF78079
:10037300DC3134E75EF709E75FF7223134E74EF704
:1003830009E74FF7223134E76EF709E76FF722C326
:10039300B24AA98019E497F709E497F780AFD380AD
:1003A300F1A980E7A2E7B04440E522204AE122A96F
:1003B300801907B70002090722C2D5A980E76005A3
:1003C300EF6002D2D519E78FF0A430D202D2D5095B
:1003D300C78EF0A430D202D2D527F772D592D519A1
:1003E300E78EF0A4F7E5F00927F772D572E792D20A
:1003F30022C24A71A4313471A471BC715071AE220E
:10040300D24C8002C24CD24A71A471923134EE4F65
:10041300604DA24AB04C924A71A4F50919E7F50858
:10042300E4F50BF50A7D11C38017E50A33F50AC518
:100433000B33C50B2EF50CE50B3F5005850C0AF568
:100443000BE50833F508E50933F509DDDD204C0735
:10045300A70809A7098005A70A09A70B71AE22619E
:1004630057AE0DAF0E314C7E557F6271BC7E197F46
:1004730036A98019715A3134BE0007BF80047E2A21
:100483007F318E0D8F0E314C2231343146F5F0A978
:100493008019C3E79E09C72044066480CF6480CFD8
:1004A3009F477004A2F180084004A2F08002A2F2E8
:1004B300E4F73319F722C2492041057A0078342240
:1004C3002042057A0C7829227A10788022882C8A97
:1004D3002D8C2E22AA2DA82CAC2E22204302E622FC
:1004E30020410EC083C0828A838882E0D082D08379
:1004F30022E8C582CAC583F8E493C8C583CAC58206
:10050300C82210490991DEFC08B800010A22EC2236
:100513002041068B838982F0222115B11309B9008A
:10052300010B22B105642060FAD249D322B105B18F
:1005330005B105B40DFB22D083D082B10591D0E47F
:1005430093A2E7547F6C7012A3400BB105BC2EEF4E
:10055300E493A330E7FAB126E473E493A330E7FA14
:1005630091D7D249C3E473B10524BFFE24E65004F6
:10057300D249C32291D0B10524BF24E65003BC2E37
:100583004091D7D249B13A44425954C550053173C9
:10059300018027B13A524249D45005317302801A7F
:1005A300B13A58425954C55005317303800CB13ADE
:1005B30043425954C55008317304120B99D322C3D3
:1005C300223173007F00314CD249A126B10551FD80
:1005D3004003D24922B105710A40FA314CD249A1F4
:1005E30026B105F5086422600864056004C3D24996
:1005F30022B105B50802A12611AFB40DF42129B12A
:1006030005BC3A0322B105BC0D0122D2492129B10F
:1006130005BC3A0122BC0D0122D249D322B105F512
:1006230030B105F52FE530A2E72230430280EED347
:100633002211ADBC3A05B1260208B40208AFE58029
:100643002404F508A8083100BE1192B41212310037
:100653008D882CA808E8652C60EFE611AF0880F5BB
:10066300B418063100238D80DBB47F11E8B508058B
:1006730031008780D431000820881880CCB8DA058F
:1006830031008780C4F611AF08B40DBDA808C24974
:1006930022C24A71A43134D248E4F5087D102044C3
:1006A3001D304A033100ADCE33CECF33CFC508352D
:1006B300E0D4C50835E0D4DDEEFFEE33AE0811E13A
:1006C300EFC411E1EF11E1304402C248EEC411E17D
:1006D300C248EE11E13044033100C822D120401258
:1006E300AF30AE2FC24AD19A3100A0B10511AFB4D9
:1006F3000DF922D24391B911CC4004D1DF50F8C295
:100703004322C24A31003AA0119211AFB4200280B1
:10071300F7B42B0280F2B42D04B24A80EB51FD50A2
:1007230007119211AFB47F063100238D80D4710A73
:1007330040EF314C61AEE4F528F529758300F5826D
:10074300745AF0E0645A600AE47810F608B828FB9B
:10075300800BD240E4F88882F008B834F922F139EA
:1007630075823474FFF02275808091B9D24322D20E
:100773004391B9313491D0D1204012EE952FF52F0A
:10078300EF9530452F60064004B13480E881D7A946
:100793002CAB2DB130B105B11E20E70DB105B11E53
:1007A300B105B11EB40DF980EC2291D7C249B10550
:1007B30020E709B105B105B40DFB80F2E50F240371
:1007C30028F9E43AFBB40702211E91E3B113E8B51B
:1007D3002C05EAB52D012218B8FF011A19B9FFEA51
:1007E3001B80E7A92CAB2DEFB11EEEB11EA82AE6A4
:1007F300B11E08B40DF92218882AF17240031207BA
:1008030092A92A1909E7B40DFBE9C3952AF50F60EC
:10081300061207AD1207E6C24322120134EE132279
:10082300120772400201AF020115AF30AE2F020171
:100833004C1207721205308073E8C0E0E58024FE95
:10084300F924F9F87D03E76670201819DDF8D0E084
:10085300F8120238E58024FDF9C3E7950809E7207B
:1008630044056480630980950922D0E0F8020129D8
:10087300C243801FA98087F019E7198980C0E0C0AF
:10088300F043D01822020129120761C24375813057
:100893007580801201004F4B8D12064112052612FE
:1008A30005CF500D1207FA80F012076A12062D4089
:1008B300DA1200CC12052612056A500812053ABD59
:1008C300502E801312053A4C45D4503012056A500D
:1008D300B412053ABD50AE51FD12053AAC500812A0
:1008E30002341203B280F0120602120238020636F4
:1008F30012060212029E12069402063412053A47A9
:100903004F54CF500751FD120608012312053A47F1
:100913004F5355C25009112D51FD120608012312E0
:10092300053A5052494ED45043120612503812051C
:100933003ABB500280F812053AAC50051200DA8037
:10094300ED12061250231205E4400551FD120694E0
:1009530012053AAC50051200DA80D312053ABB50A7
:100963000280CB12060202063402063612053A4909
:10097300C6501651FD12053A544845CE5000111D7C
:10098300500201B412053401AF12053A494E5055D5
:10099300D4502B1205E4400B12056A5019120705B7
:1009A30012023812053ABB500280E812053AAC50E5
:1009B300071200DA80DD61DC12060202063412053A
:1009C3003A5245545552CE500512060801341205C9
:1009D3003A43414CCC500D51FD120608117753D0C8
:1009E300E702063612053A464FD2502112056A50E5
:1009F3004B12053ABD504551FD12023412053A54CB
:100A0300CF503951FD120608112D02063612053A50
:100A13004E4558D4502812056A502112060212027C
:100A23009A1203B2113C400512015F0134120134E2
:100A330012013412013412014602063601881205EE
:100A43003A454EC45005120608017312053A4C4943
:100A530053D45014120612500A51FD120772120693
:100A6300FA01961206F6019612053A5255CE500532
:100A730012060801AC12053A4E45D750051206027C
:100A8300018B12053A52455345D450061206020211
:100A9300000012053A524FCD500A120602D241C24B
:100AA3004202063612053A5241CD5008120602C2DE
:100AB3004102063612053A50524FCD500A12060231
:100AC300D241D24202063612053A4845D85008129E
:100AD3000602D24402063612053A444543494D41C3
:100AE300CC5008120602C24402063612053A524599
:100AF300CD500512053401AF0188710A71DE5040F3
:100B0300710A12048C80F5714412053AAB500771D7
:100B13004412036280F312053AAD50077144120385
:100B23006880E612053A4FD25007714412037E8063
:100B3300D812053A584FD25007714412038880C91E
:100B430022717F12053AAA5007717F1203F480F3D2
:100B530012053AAF5007717F12040780E612053A77
:100B6300414EC45007717F12037480D712053A4D6A
:100B73004FC45007717F12040380C82212053AAD97
:100B8300500671991203922212053A4E4FD4500621
:100B930071991203A12212056A500412029E2212B5
:100BA30005CF50012212053A524EC4500F1204646D
:100BB30071CD1204031203A41203B22212053A41A7
:100BC30042D3500671CD1203A42212053AA850094C
:100BD30051FD12053AA9500122018812053ABD5070
:100BE30005120173022212053A3CBD50051201732E
:100BF300062212053A3CBE50051201730522120566
:100C03003ABC5005120173042212053A3EBD500549
:100C1300120173032212053ABE5005120173012219
:100C2300C3220F8F9022000A464F5220493D3120A4
:100C3300544F20390D0014464F52204A3D31205461
:100C43004F20390D001E5052494E5420492A4A2C38
:100C53000D00284E455854204A0D00325052494E3B
:0C0C6300540D003C4E45585420490D80B3
:00000001FF
